:100000000C94DD020C9405030C9405030C94050379
:100010000C9405030C9405030C9405030C94050340
:100020000C9405030C9405030C9405030C94050330
:100030000C9405030C9405030C9405030C94050320
:100040000C94D30B0C9405030C94430C0C941D0CD2
:100050000C9405030C9405030C9405030C94050300
:100060000C9405030C940503000000080002010035
:100070000003040700000000000000000000000072
:10008000003E5B4F5B3E3E6B4F6B3E1C3E7C3E1C1E
:10009000183C7E3C181C577D571C1C5E7F5E1C0064
:1000A000183C1800FFE7C3E7FF0018241800FFE71B
:1000B000DBE7FF30483A060E2629792926407F05DE
:1000C0000507407F05253F5A3CE73C5A7F3E1C1CF4
:1000D00008081C1C3E7F14227F22145F5F005F5FB4
:1000E00006097F017F006689956A606060606094A0
:1000F000A2FFA29408047E040810207E20100808A5
:100100002A1C08081C2A08081E101010100C1E0CAF
:100110001E0C30383E3830060E3E0E060000000041
:100120000000005F00000007000700147F147F1428
:10013000242A7F2A1223130864623649562050006D
:1001400008070300001C2241000041221C002A1C59
:100150007F1C2A08083E0808008070300008080844
:100160000808000060600020100804023E51494564
:100170003E00427F400072494949462141494D3382
:100180001814127F1027454545393C4A49493141E9
:10019000211109073649494936464949291E0000B7
:1001A000140000004034000000081422411414140C
:1001B0001414004122140802015909063E415D59F8
:1001C0004E7C1211127C7F494949363E4141412201
:1001D0007F4141413E7F494949417F090909013E2B
:1001E000414151737F0808087F00417F4100204052
:1001F000413F017F081422417F404040407F021C64
:10020000027F7F0408107F3E4141413E7F0909097A
:10021000063E4151215E7F09192946264949493246
:1002200003017F01033F4040403F1F2040201F3F0C
:100230004038403F63140814630304780403615991
:10024000494D43007F4141410204081020004141D3
:10025000417F04020102044040404040000307087F
:100260000020545478407F2844443838444444287B
:10027000384444287F385454541800087E09021822
:10028000A4A49C787F0804047800447D40002040AA
:10029000403D007F1028440000417F40007C0478EE
:1002A00004787C080404783844444438FC18242436
:1002B0001818242418FC7C080404084854545424B6
:1002C00004043F44243C4040207C1C2040201C3C33
:1002D0004030403C44281028444C9090907C44642A
:1002E000544C4400083641000000770000004136BD
:1002F000080002010204023C2623263C1EA1A16143
:10030000123A4040207A3854545559215555794174
:100310002254547842215554784020545579400C49
:100320001E5272123955555559395454545939552C
:100330005454580000457C410002457D420001456F
:100340007C407D1211127DF0282528F07C54554503
:10035000002054547C547C0A097F4932494949326F
:100360003A4444443A324A4848303A4141217A3A80
:1003700042402078009DA0A07D3D4242423D3D404C
:1003800040403D3C24FF2424487E4943662B2FFCFB
:100390002F2BFF0929F620C0887E090320545479A9
:1003A000410000447D413048484A32384040227A7A
:1003B000007A0A0A727D0D19317D2629292F2826F7
:1003C0002929292630484D402038080808080808FF
:1003D0000808382F10C8ACBA2F102834FA00007B58
:1003E000000008142A142222142A1408550055006B
:1003F00055AA55AA55AAFF55FF55FF000000FF005A
:10040000101010FF00141414FF001010FF00FF1054
:1004100010F010F0141414FC001414F700FF000086
:10042000FF00FF1414F404FC141417101F10101F05
:10043000101F1414141F00101010F0000000001FF3
:10044000101010101F10101010F010000000FF10FE
:100450001010101010101010FF10000000FF1400FA
:1004600000FF00FF00001F10170000FC04F414142C
:100470001710171414F404F40000FF00F7141414F8
:1004800014141414F700F7141414171410101F1078
:100490001F141414F4141010F010F000001F101F9B
:1004A0000000001F14000000FC140000F010F01009
:1004B00010FF10FF141414FF141010101F00000080
:1004C00000F010FFFFFFFFFFF0F0F0F0F0FFFFFF84
:1004D0000000000000FFFF0F0F0F0F0F38444438DB
:1004E00044FC4A4A4A347E02020606027E027E022A
:1004F00063554941633844443C04407E201E200635
:10050000027E020299A5E7A5991C2A492A1C4C7271
:1005100001724C304A4D4D303048784830BC625AF8
:10052000463D3E494949007E0101017E2A2A2A2A88
:100530002A44445F444440514A444040444A514064
:100540000000FF0103E080FF000008086B6B083625
:1005500012362436060F090F060000181800000096
:100560001010003040FF0101001F01011E00191D85
:100570001712003C3C3C3C00000000000000000062
:10058000250028002B0000000000240027002A007E
:100590000404040404040404020202020202030329
:1005A0000303030301020408102040800102040831
:1005B0001020010204081020750C11241FBECFEF7B
:1005C000D8E0DEBFCDBF13E0A0E0B1E0E4E0FCE1A5
:1005D00002C005900D92A633B107D9F724E0A6E337
:1005E000B3E001C01D92A730B207E1F712E0CDEDF4
:1005F000D2E004C02197FE010E94F50DCC3DD10749
:10060000C9F70E94D10C0C94000E0C94000090913C
:10061000F8039F3F21F49091F9039F3F59F128E09F
:1006200030E040E8E0910304F0910404508190919F
:100630000604909595239083E0910104F0910204C3
:1006400090910504582F542319F05081952B03C025
:100650005081909595239083E0910304F0910404D8
:10066000508190910604952B908346952150310935
:10067000C9F608958EBD00000DB407FEFDCF8EB5FE
:10068000089590E0FC01EC55FA4F2491FC01E057ED
:10069000FA4F8491882399F090E0880F991FFC010C
:1006A000EA57FA4FA591B491FC01E458FA4F8591AD
:1006B00094918FB7F894EC91E22BEC938FBF08954F
:1006C0002F923F924F925F926F927F928F929F9262
:1006D000AF92BF92CF92DF92EF92FF920F931F9350
:1006E000CF93DF93CDB7DEB76B970FB6F894DEBF2D
:1006F0000FBECDBF9B8F8A8F1B014A01D22E198757
:1007000008873701A982DC0159962D913C915A97AF
:100710002115310509F0FFC018968D919C9119970C
:10072000681779070CF0E7C11A968D919C911B9779
:10073000481759070CF0DFC1EC2DF0E0FB83EA838A
:100740009B0146E0C49E200D311D11243D872C875E
:10075000121613060CF0CFC16A2D70E07B876A87F2
:1007600083E0660F771F8A95E1F77F876E87CB015D
:10077000880D991D181619060CF0BDC158968C915C
:10078000811104C08FEA8D1508F4D394AA8DBB8D16
:10079000ED91FC9111970284F385E02DCD0109952F
:1007A000B5E0DB9EC0011124EC2DF0E0F98BE88B65
:1007B00091012B5F3F4F3B8B2A8B3D822C82210185
:1007C000AC01421953095D8B4C8B7981672F70E026
:1007D0007F8B6E8BC4010896998F888FEC89FD8979
:1007E000E40DF51DE458FF4FD49054019F828E8292
:1007F000D0FE16C0AA8DBB8DED91FC91B1E0CB125D
:1008000009C02981213031F40484F585E02D288543
:10081000398519C00684F785E02DE884F9841DC068
:10082000488559854615570519F1AA8DBB8DED915F
:10083000FC91B1E0CB120DC02981213051F4048428
:10084000F585E02D9301A501B2018A8D9B8D099557
:100850000FC00684F785E02D73010A851B852A8168
:100860003B814E815F816C817D818A8D9B8D099555
:10087000D6943FEFA31AB30A4E815F816E897F89B8
:10088000460F571F5F834E83888D998DA816B90632
:1008900009F0AECF9FEF491A590AAC81BD81E889B2
:1008A000F989AE0FBF1FBD83AC832A893B894216ED
:1008B000530609F093CF488559854615570509F425
:1008C000F8C0AA8DBB8DED91FC91B1E0CB1211C0A7
:1008D0002981213071F4B1016B5F7F4F0088F1896C
:1008E000E02D830128E030E0A4018A8D9B8D0995DD
:1008F000E0C06C857D854A815B81641B750B068435
:10090000F785E02D73010E851F859A01A4018A8D5C
:100910009B8D0995CEC0F9013496E491DE1AF90158
:10092000329685919491B7E0DB9E800D911D112444
:10093000F901259134913B8B2A8BFC01259134914F
:100940005901FC0132965490319634913C8732968D
:1009500074903196149141E04C1518F05981523041
:1009600068F0672D072C000C770B7D836C83812F3B
:10097000012E000C990B9B838A8304C01B821A8270
:100980001D821C82AA8DBB8DED91FC911197028472
:10099000F385E02DCD010995412CD12C612CF981F5
:1009A000EF2FF0E0FF83EE832C2D30E03B872A878A
:1009B000A401410F511D17FD5A955F8B4E8BB1015C
:1009C000670D711D77FC7A95798F688F7C85671626
:1009D00008F06FC0262D30E04A815B81420F531F23
:1009E000AE81BF81A49FC001A59F900DB49F900DC3
:1009F0001124F401E80FF91FF98BE88B842D712C79
:100A00004E895F89420F531F5D8B4C8B751408F024
:100A10004DC051E0580F5E87877041F4C5010196C3
:100A2000EA89FB89EA0DFB1DD4905C01D7FE3AC030
:100A300061E0C61216C07981713099F4AA8DBB8D20
:100A4000ED91FC9111970484F585E02D2885398579
:100A50004C895D89688D798D670D711DCD01099572
:100A600021C08C819D81870D911DEA85FB858E9F1C
:100A7000B0018F9F700D9E9F700D1124620D731D2C
:100A8000AA8DBB8DED91FC9111970684F785E02D21
:100A9000E884F9840E811F812A853B85488959891C
:100AA000CD010995DD0C73948E85B0CF450C639410
:100AB0008DCFAA8DBB8DED91FC9111970688F7899A
:100AC000E02DCD016B960FB6F894DEBF0FBECDBF03
:100AD000DF91CF911F910F91FF90EF90DF90CF901A
:100AE000BF90AF909F908F907F906F905F904F904E
:100AF0003F902F9009946B960FB6F894DEBF0FBE0F
:100B0000CDBFDF91CF911F910F91FF90EF90DF90BC
:100B1000CF90BF90AF909F908F907F906F905F909D
:100B20004F903F902F90089590E0FC01E859FF4FBF
:100B30002491FC01EC55FA4F3491FC01E057FA4F37
:100B4000E491EE2309F43CC0222339F1233091F0E3
:100B500038F42130A9F0223001F584B58F7D12C020
:100B6000273091F02830A1F02430B9F48091800032
:100B70008F7D03C0809180008F77809380000DC0AF
:100B800084B58F7784BD09C08091B0008F7703C092
:100B90008091B0008F7D8093B000F0E0EE0FFF1FDA
:100BA000E458FA4FA591B4919FB7F894611104C02D
:100BB0008C913095382302C0EC913E2B3C939FBF23
:100BC0000895CF93C82F60E08091FA030E949405A6
:100BD0008091FC0318161CF460E00E9494058C2F91
:100BE0000E9407038091FC03181624F461E0CF9162
:100BF0000C949405CF910895CF93C82F87FDCFE72C
:100C0000C093FD0381E20E94E1058C2F80680E9461
:100C1000E10580E2CF910C94E1053FB7F894809113
:100C20003C0390913D03A0913E03B0913F0326B554
:100C3000A89B05C02F3F19F00196A11DB11D3FBF14
:100C4000BA2FA92F982F8827820F911DA11DB11DA2
:100C5000BC01CD0142E0660F771F881F991F4A959E
:100C6000D1F708958F929F92AF92BF92CF92DF9269
:100C7000EF92FF926B017C010E940D064B015C011B
:100C8000C114D104E104F104F1F00E940D06DC016D
:100C9000CB0188199909AA09BB09883E9340A1058F
:100CA000B10570F321E0C21AD108E108F10888EE1D
:100CB000880E83E0981EA11CB11CC114D104E1046C
:100CC000F10419F7DDCFFF90EF90DF90CF90BF9048
:100CD000AF909F908F900895CF938091FB0318164B
:100CE00074F460E00E94940564EF71E080E090E0AD
:100CF0000E94320661E08091FB030E949405C0913E
:100D0000FE03C83008F0C7E0C093FE0381E20E94F2
:100D1000E1058C2F80610E94E10580E20E94E105DF
:100D20008091FD030E94FC0580E20E94E1058CE0B9
:100D3000CF910C94E105EF92FF920F931F93CF9305
:100D4000DF939091FF03992361F0809100048F5FFE
:100D5000891718F48093000404C0109200040E94C4
:100D60006C0600E011E0C0E08C2F80640E94E10579
:100D700080E80E94E10561E08091FA030E949405F9
:100D80008091FC0318161CF460E00E949405780121
:100D9000D4E5F70181917F010E940703D150C9F783
:100DA0008091FC0318161CF461E00E949405CF5F4B
:100DB0000C5A1F4FC630C1F680E4DF91CF911F91CE
:100DC0000F91FF90EF900C94E105CF92DF92EF929C
:100DD000FF920F931F93CF93DF936C017A018B01E6
:100DE000C0E0D0E0CE15DF0581F0D8016D918D0116
:100DF000D601ED91FC910190F081E02DC60109959D
:100E0000892B11F02196EECF7E01C701DF91CF91A2
:100E10001F910F91FF90EF90DF90CF900895FC010C
:100E2000538D448D252F30E0842F90E0821B930B4F
:100E3000541710F0CF96089501970895FC01918DF5
:100E4000828D981761F0828DDF01A80FB11D5D962C
:100E50008C91928D9F5F9F73928F90E008958FEF9A
:100E60009FEF0895FC01918D828D981731F0828D4E
:100E7000E80FF11D858D90E008958FEF9FEF0895A5
:100E8000FC01918D228D892F90E0805C9F4F821B09
:100E900091098F739927089580E493E00E94400799
:100EA00021E0892B09F420E0822F0895FC01848D34
:100EB000DF01A80FB11DA35ABF4F2C91848D90E084
:100EC00001968F739927848FA689B7892C93A0895F
:100ED000B1898C91837080648C93938D848D9813E9
:100EE00006C00288F389E02D80818F7D808308957C
:100EF000EF92FF920F931F93CF93DF93EC0181E06A
:100F0000888F9B8D8C8D981305C0E889F989808125
:100F100085FD26C0F62E0B8D10E00F5F1F4F0F735F
:100F20001127E02E8C8DE8120CC00FB607FCFACF0B
:100F3000E889F989808185FFF5CFCE010E945607A7
:100F4000F1CF8B8DFE01E80FF11DE35AFF4FF082C8
:100F50009FB7F8940B8FEA89FB89808180620AC071
:100F60009FB7F894EE89FF896083E889F9898081C9
:100F70008370806480839FBF81E090E0DF91CF9198
:100F80001F910F91FF90EF900895CF93DF93EC01A5
:100F9000888D8823C9F0EA89FB89808185FD05C099
:100FA000A889B9898C9186FD0FC00FB607FCF5CFD3
:100FB000808185FFF2CFA889B9898C9185FFEDCF1B
:100FC000CE010E945607E7CFDF91CF91089580E0D0
:100FD00090E0892B29F00E944C0781110C940000AD
:100FE0000895FC0177FD68C08085918568177907B1
:100FF0000CF062C057FD60C0828593854817590781
:101000000CF05AC08689823059F08330B1F08130BB
:10101000D1F48FE290E0861B970BBA01AC0113C0AC
:1010200083E590E0FC01E61BF70BBF018FE290E047
:10103000FC01E41BF50BAF0106C083E590E0841BC7
:10104000950BAB01BC0164357105B0F5403351051A
:1010500098F5CA01E3E095958795EA95E1F7477021
:101060005527232BA1F024E5289FF001299FF00D9F
:1010700011246E0F7F1FFB01E050FF4F81E090E0D5
:1010800001C0880F4A95EAF79081892B14C024E5A6
:10109000289FF001299FF00D11246E0F7F1FFB0187
:1010A000E050FF4F81E090E001C0880F4A95EAF7D9
:1010B000809590818923808308950895FC01637051
:1010C000668B8481958126813781613039F0633068
:1010D00029F0918780873387228708953187208779
:1010E0009387828708958F929F92AF92CF92EF92CB
:1010F000FF920F931F93CF93DF93EC01262F898DDF
:101100009A8D009709F042C06A3059F41D861C86FA
:101110002D898E859F8538E0239F800D911D112498
:1011200043C06D3009F4AAC08F898823C9F03C8977
:101130008C859D8546E0349F800D911D1124488546
:1011400059854817590764F41D861C863D898E858C
:101150009F8548E0349F800D911D11249F878E87C5
:10116000EA88FB88088919894E855F856C857D85AD
:10117000AD88CC88CE010E9460032C898C859D852A
:1011800036E0239F800D911D11243EC06A3079F412
:101190001D861C862D89FC013696E4918E859F85DF
:1011A0002E9F800D911D11249F878E8767C06D3003
:1011B00009F464C0FC0134963491631708F45EC0EE
:1011C0003196E491E61708F459C0462F431B342F9B
:1011D000FC0132968590949047E0349F800C911CDE
:1011E0001124F401329634913196E491332311F0B5
:1011F000E1110DC0F4013496E4912C898C859D8514
:10120000E29F800D911D11249D878C8737C0F401CA
:10121000359644915F89552319F15C89E32FF0E0FD
:10122000E40FF11D47FDFA955E9FB0015F9F700DC1
:1012300011244C855D85460F571F68857985641795
:10124000750774F41D861C863D89FC013696E49171
:101250008E859F853E9F800D911D11249F878E87CF
:10126000EA88FB88088919894E855F856C857D85AC
:10127000AD88CC88CE010E946003BCCF81E090E0B5
:10128000DF91CF911F910F91FF90EF90CF90AF9092
:101290009F908F9008956F927F928F929F92AF92BE
:1012A000BF92CF92DF92EF92FF920F931F93CF9353
:1012B000DF93EC014B015A0169013801E881F981A2
:1012C0000284F385E02D0995E881F9810288F3898C
:1012D000E02D87019601A501B401CE010995A50174
:1012E000460D571D41505109E881F9810288F38963
:1012F000E02D9601B401CE010995E881F9810088BD
:10130000F189E02D9301A501B401CE010995C80C26
:10131000D91CB60161507109E881F9810088F18911
:10132000E02D9301A501CE010995E881F981068898
:10133000F789E02DCE01DF91CF911F910F91FF90A2
:10134000EF90DF90CF90BF90AF909F908F907F9065
:101350006F9009948F929F92AF92BF92CF92DF923B
:10136000EF92FF920F931F93CF93DF934C016B018A
:101370005A01E901DC01ED91FC916217730781F4D8
:101380000417150724F48B2D5801042F182F0A1960
:101390001B0998012F5F3F4F048CF58DE02D12C083
:1013A0004017510709F52617370724F48D2D6901D9
:1013B000C62FD82F9E012C193D092F5F3F4F068C59
:1013C000F78DE02D8701A501B601C4010995DF91D4
:1013D000CF911F910F91FF90EF90DF90CF90BF9032
:1013E000AF909F908F9008950284F385E02D09952A
:1013F000D401ED91FC910488F589E02D9E01A501B1
:10140000B601C4010995D401ED91FC910688F789D4
:10141000E02DC401DF91CF911F910F91FF90EF90CC
:10142000DF90CF90BF90AF909F908F900994EF92F4
:10143000FF920F931F93DC011A960D911C911B973D
:1014400018962D913C911997ED91FC9100A0F1A176
:10145000E02D7B0140E050E060E070E009951F91D5
:101460000F91FF90EF9008954F925F926F927F924D
:101470008F929F92AF92BF92CF92DF92EF92FF92A4
:101480000F931F93CF93DF936C012B015A01390106
:101490004801DC01ED91FC910284F385E02D099572
:1014A000E201640C751CD601ED91FC91C615D705BF
:1014B0005CF40088F189E02D87019401A501BE014B
:1014C000C60109952196EFCF0688F789E02DC60160
:1014D000DF91CF911F910F91FF90EF90DF90CF9010
:1014E000BF90AF909F908F907F906F905F904F9044
:1014F00009948F929F92AF92BF92CF92DF92EF9218
:10150000FF920F931F93CF93DF93EC015B014A018E
:101510006901E881F9810284F385E02D099595013F
:101520002C0D3D1D21503109E881F9810488F58990
:10153000E02D78018401A401B501CE010995E8816F
:10154000F9810688F789E02DCE01DF91CF911F91B7
:101550000F91FF90EF90DF90CF90BF90AF909F9052
:101560008F9009948F929F92AF92BF92CF92DF9209
:10157000EF92FF920F931F93CF93DF93EC015B01E8
:101580004A0169017801E881F9810284F385E02D3F
:101590000995C80CD91C860101501109E881F9810F
:1015A0000488F589E02D9501A401B501CE010995C6
:1015B000E881F9810688F789E02DCE01DF91CF918E
:1015C0001F910F91FF90EF90DF90CF90BF90AF9061
:1015D0009F908F9009940895EF92FF920F931F931D
:1015E000DC01ED91FC9100A0F1A1E02D09951F9186
:1015F0000F91FF90EF9008950F931F93DC01ED91F1
:10160000FC91068CF78DE02D09951F910F9108959F
:101610000F931F93DC01ED91FC91048CF58DE02D6F
:1016200009951F910F910895DC01ED91FC910084C3
:10163000F185E02D09942F923F924F925F926F9225
:101640007F928F929F92AF92BF92CF92DF92EF9252
:10165000FF920F931F93CF93DF9300D000D000D061
:10166000CDB7DEB72C017E836D836A015901C801B5
:10167000FC82EB824801841A950A97FE03C091947C
:101680008194910835012D813E81621A730A77FE9B
:1016900003C0719461947108681479045CF43A2D64
:1016A0002B2D5C01832F922F3D812E81DE82CD82F6
:1016B000C32ED22EAD81BE81AA16BB065CF43C2D92
:1016C0002D2D6C01832F922F3D812E81BE82AD8204
:1016D000A32EB22E85012D813E81021B130B1C010E
:1016E0002C183D0837FE03C031942194310878014D
:1016F00017FF03C03FEFE31AF30AF594E794C81607
:10170000D9062CF08FEF9FEF9A83898304C0A1E064
:10171000B0E0BA83A9832D813E81A216B30624F1DD
:10172000D201ED91FC910484F585E02D2B813C8163
:101730006814790424F44D815E81B60103C0A601CA
:101740006D817E81C2010995E218F308F7FE06C09B
:1017500029813A81C20ED31EE00EF11E8D819E8139
:1017600001969E838D83D7CF26960FB6F894DEBF61
:101770000FBECDBFDF91CF911F910F91FF90EF90E2
:10178000DF90CF90BF90AF909F908F907F906F90A1
:101790005F904F903F902F900895089580E090E0E3
:1017A00008950E94FB0D1F920F920FB60F92112405
:1017B0002F933F938F939F93AF93BF938091380361
:1017C00090913903A0913A03B0913B0330913703D4
:1017D00023E0230F2D3720F40196A11DB11D05C074
:1017E00026E8230F0296A11DB11D20933703809395
:1017F000380390933903A0933A03B0933B0380914D
:101800003C0390913D03A0913E03B0913F030196AC
:10181000A11DB11D80933C0390933D03A0933E0313
:10182000B0933F03BF91AF919F918F913F912F91C3
:101830000F900FBE0F901F9018951F920F920FB62A
:101840000F9211242F933F934F935F936F937F9346
:101850008F939F93AF93BF93EF93FF9380E493E0B5
:101860000E945607FF91EF91BF91AF919F918F9189
:101870007F916F915F914F913F912F910F900FBE8C
:101880000F901F9018951F920F920FB60F92112470
:101890002F938F939F93EF93FF93E0915003F091D9
:1018A00051038081E0915603F091570382FD12C0ED
:1018B0009081809159038F5F8F7320915A03821713
:1018C00051F0E0915903F0E0E05CFC4F958F80937C
:1018D000590301C08081FF91EF919F918F912F91CA
:1018E0000F900FBE0F901F901895E0E4F3E0138265
:1018F000128288EE93E0A0E0B0E084839583A68313
:10190000B7838CEF92E09183808385EC90E095879C
:10191000848784EC90E09787868780EC90E0918BB9
:10192000808B81EC90E0938B828B82EC90E0958BA6
:10193000848B86EC90E0978B868B118E128E138EA3
:10194000148EEDEDF3E01382128224E530E035834E
:10195000248380E390E09783868331872087938771
:101960008287168A158614861786168681E0858BEF
:10197000848B2FEF3FEF338B228B318B208B878B28
:10198000108E128E118E8EE093E0918380838FEF04
:10199000838F848F85E0858F83E0868F84E0878FB7
:1019A0000895789484B5826084BD84B5816084BDD7
:1019B00085B5826085BD85B5816085BD80916E00ED
:1019C000816080936E00109281008091810082601E
:1019D000809381008091810081608093810080915B
:1019E00080008160809380008091B100846080934A
:1019F000B1008091B00081608093B00080917A0046
:101A0000846080937A0080917A00826080937A006B
:101A100080917A00816080937A0080917A0080685A
:101A200080937A001092C100E0915003F09151032D
:101A300082E08083E0914C03F0914D031082E091AD
:101A40004E03F0914F038FEC808310925803E09186
:101A50005403F091550386E08083E0915203F091A6
:101A60005303808180618083E0915203F09153039E
:101A7000808188608083E0915203F09153038081DC
:101A800080688083E0915203F091530380818F7DC1
:101A900080838091F8038F3F29F49091F9039F3F51
:101AA00009F466C00E9441038091F9030E9441033A
:101AB0008091F903082E000C990BFC01E057FA4FB6
:101AC000E491F0E0EE0FFF1FE458FA4F25913491B6
:101AD0003093040420930304FC01EC55FA4FE49185
:101AE000E09306048091F803082E000C990BFC018A
:101AF000E057FA4FE491F0E0EE0FFF1FE458FA4F81
:101B0000259134913093020420930104FC01EC559B
:101B1000FA4FE491E09305048091FA030E94410397
:101B20008091FB03181614F40E9441038091FC037A
:101B3000181614F40E94410384E08093FE0388E2A7
:101B40008093FD031092FF03109200040E946C0624
:101B50000E949B0682E30E94FC050E949B0660EDAA
:101B600077E080E090E00E9432060E94E707FDCF18
:101B7000CFB7F89480913603811124C0EAE9F5E0EB
:101B80008491EEEAF5E09491E82FF0E0EE0FFF1F6C
:101B9000EA57FA4FA591B491EC91E92321F461E061
:101BA0008AE00E9494058AE00E9441038CB580611E
:101BB0008CBD8CB580648CBD8DE00E9441038BE0B0
:101BC0000E944103809136038F5F80933603CFBF1D
:101BD0008CB58C7F8CBD8DB58E7F8DBD8CB5837F94
:101BE0008CBD8CB58F7D8CBD97CFEE0FFF1F059000
:101BF000F491E02D099481E090E0F8940C94000EAB
:101C040000000000000000000000000000000000D0
:101C140000000000000000000000000000000000C0
:101C2400000000000000C0E0F0F8FCFCFEFFFCE057
:101C340000000000000000000000000000000000A0
:101C44000000000000000000000000000000000090
:101C54000000000000000000000000000000000080
:101C64000000000000F8F8F8F8F8F8F8F8F8F8F8C8
:101C7400F8F0F0E0E0C080C0FCFFFFFFFF7F3F7F93
:101C8400FFFFFFFFFF000000000000000000000055
:101C94000000000000000000000000000000000040
:101CA4000000000000000000000000000000000030
:101CB400000000000000000000000F1F3F7FFFFF36
:101CC400FFFFFFFFFFFFE7C7C7878F9F9FFFFFFF50
:101CD400C1C0E0FCFFFFFFFFFFFCFCFCFCFEFEFEBE
:101CE400FCFCF8F8F0E0C0C00000000000000000B8
:101CF40000000000000000000000000000000000E0
:101D040000000000000000000000000000000000CF
:101D14000080C0E0F1FBFFFFFFFFFF7F1F0F0F8775
:101D2400E7FFFFFF1F1F3FF9F8F8F8F8F8F8FDFF89
:101D3400FFFFFFFFFFFFFFFF7F3F0F0701000000D2
:101D4400000000000000000000000000000000008F
:101D5400000000000000000000000000000000007F
:101D6400000000F0FEFFFFFFFFFFFFFFFFFFFFFE8D
:101D74007E3F3F0F1FFFFFFFFCF0E0F1FFFFFFFF7F
:101D8400FFFCF0010101010101010100000000005C
:101D9400000000000000000000000000000000003F
:101DA400000000000000000000000000000000002F
:101DB4000000000000000003030303030303030106
:101DC40001010100000000000000030F1F3F7F7F9E
:101DD400FFFFFFFF7F7F1F030000000000000000E3
:101DE40000000000000000000000000000000000EF
:101DF4000000000000000000000000007807E50675
:101E04000F07C50740071E073207000000007308CC
:101E1400E506CE0BCD0BF107EB0A140BEC0A080B0D
:101E2400FC0A1B0BEB0A5E085D08B20A790A340A45
:061E3400170AAA094B0980
